:100000000206C3E524544024C070030201B9244011
:100010006003020205E52454F824E8606624F870C1
:100020000302016F24F8700302019A24F87003029E
:1000300001A524F870030201AE2428600302020522
:10004000E524540724FC601714601B14601E146020
:1000500026240460030202057F01120FCF801BE4F7
:10006000FF120FCF8009120F598F3B22120D70AC77
:1000700006AD077F018009120D70AC06AD07E4FFE5
:10008000020F9AE5245407B40800400302020590C9
:100090000096F82828730200AE0200B30200B902ED
:1000A00000C90200E102010802012D02014E120DF9
:1000B00070807F120D70020153E4FF120FCF7C009D
:1000C000EF253BFDEC3EFC806D7F02120FCF7C00E4
:1000D000EF253BFDEC3EFC7F03120F9A900003805E
:1000E00069120D70AC06AD077F03120F9A7F0312E1
:1000F0000FCF74002FF58274003EF583E02400F5E5
:1001000082E43400F5838042120D70AC06AD077FA7
:1001100003120F9A7F03120FCF74002FF582740021
:100120003EF583E02400F582E43400803CE4FF12D5
:100130000FCFAC06AD077F03120F9A7F03120FCFCC
:1001400074002FF58274003EF583E0F53B22E4FF56
:10015000120FCFAC06AD077F03120F9A7F03120F69
:10016000CF74002FF58274003EF583E53BF022E466
:10017000FF120FCFAC06AD077F03120F9AE5245490
:1001800007FF120B30C0077F03120FCF74002FF54B
:100190008274003EF583D0E0F022120F59AD07E5DE
:1001A000245407805CE5245407FFAD3B8054E524CC
:1001B0005407FF120B308F3B22E5245438131313DE
:1001C000541FFFE52454076F7024FF120FCFAC06B5
:1001D000AD077F03120F9A7F03120FCF74002FF524
:1001E0008274003EF583E0FDE52454078013E52486
:1001F0005407FF120B30AD07E52454381313135482
:100200001FFF120B6822E54E60030203E112101576
:10021000EF24AC70030203DC2454B40F004003024B
:1002200003E4900229F828287302025602025902B8
:10023000025C02026E02027C02028D02029802023D
:10024000FB0203E402035E02036202036602036A26
:100250000203AF0203B30203E1020A411210158F39
:10026000261210158F27742A2526F8A62722121089
:10027000158F26742A2FF8E6FF0203DE1210158F61
:10028000261210158F27AD27AF26020E3912101532
:100290008F26120E150203DE1210158F261210156E
:1002A0008F271210158F281210158F29E526F53C7F
:1002B000E527F53D853C21853D22E528FEE52925FC
:1002C0003DFFE53C3EFEC3E5229FE5219E40030243
:1002D00003E4C3E52294FFE52194FF40030203E415
:1002E00012101574002522F58274003521F583EF74
:1002F000F00522E52270C3052180BF1210158F265C
:100300001210158F271210158F281210158F29E53E
:1003100026F53CE527F53D853C21853D22E528FE77
:10032000E529253DFFE53C3EFEC3E5229FE5219EF4
:1003300040030203E4C3E52294FFE52194FF400358
:100340000203E474002522F58274003521F583E070
:10035000FF1210190522E52270C3052180BFAF3BB3
:10036000807CAF238078AF2480741210158F261202
:1003700010158F277F02120FCF8E3C8F3D853C21B9
:10038000853D22E526FEE527253DFFE53C3EFEC3F3
:10039000E5229FE5219E504CE522F47003E521F40F
:1003A0006042120F010522E52270D8052180D47524
:1003B0004E01221210158F261210158F27121015BC
:1003C0008F28E526D39407501BE527FEE528FFE597
:1003D0002625E0243EF8A60608A607227F41021043
:1003E00019120F0122E5245407FFC39406504C1242
:1003F0000B30E53B2FFFE433FEC006C0077F07123A
:100400000E15EFFDD0E02DFFD0E03400FED3EF94C9
:10041000FFEE6480948040047D018002E4FD7F074C
:10042000120E39E5245407FF120B30E53B2FFEC0B6
:10043000067F07120E15D0E00204C8E524540724F5
:10044000F960400460030204CF120F598F3A7F070E
:10045000120E157E00E53B253AFDE433CD2FFFEE6D
:100460003DFED3EF94FFEE6480948040047D0180D4
:1004700002E4FD7F07120E397F07120E15E53B25BA
:100480003A8045E4FF120FCFAC06AD077F03120F91
:100490009A7F07120E157E00900003E0253BFDE4D5
:1004A00033CD2FFFEE3DFED3EF94FFEE64809480BA
:1004B00040047D018002E4FD7F07120E397F0712A0
:1004C0000E15900003E0253B2FF53BFF120D3D225A
:1004D000E5245407FFC39406503C120B30C3E53BA0
:1004E0009FFFC0077F07120E15C3D0E09FC3940083
:1004F00050047D018002E4FD7F07120E39E524548B
:1005000007FF120B30C3E53B9FFFC0077F07120EAA
:1005100015C3D0E08076E524540724F960310470D7
:1005200072120F598F3A7F07120E15C3E53B953AA9
:10053000C39FC3940050047D018002E4FD7F071235
:100540000E397F07120E15C3E53B953AC3803DE493
:10055000FF120FCFAC06AD077F03120F9A7F071271
:100560000E15900003E0FEC3E53B9EC39FC39400BD
:1005700050047D018002E4FD7F07120E397F0712CF
:100580000E15900003E0FEC3E53B9EC39FF53BFFC5
:10059000120D3D22E5245407FFC39406502B120B85
:1005A00030E53B2FFFE433FED3EF94FFEE648094FD
:1005B0008040047D018002E4FD7F02120E39E524B3
:1005C0005407FF120B30EF8063E524540724F960D1
:1005D00029047060120F598F3AE53B2FFFE433FE78
:1005E000D3EF94FFEE6480948040047D018002E4A8
:1005F000FD7F02120E39E53A8032E4FF120FCFACD4
:1006000006AD077F03120F9A900003E0253BFFE43D
:1006100033FED3EF94FFEE6480948040047D01802C
:1006200002E4FD7F02120E39900003E0253BF53B0A
:10063000FF120D3D22E5245407FFC39406502112FA
:100640000B30C3E53B9FC3940050047D018002E45E
:10065000FD7F03120E39E5245407FF120B3080583A
:10066000E524540724F96024047057120F598F3A77
:10067000C3E53B953AC3940050047D018002E4FD3C
:100680007F03120E39C3E53B953A8030E4FF120F29
:10069000CFAC06AD077F03120F9A900003E0FFC3B3
:1006A000E53B9FC3940050047D018002E4FD7F037D
:1006B000120E39900003E0FFC3E53B9FF53BFF12AC
:1006C0000D3D22787FE4F6D8FD75814E02070A02BF
:1006D0000F72E493A3F8E493A34003F68001F208B9
:1006E000DFF48029E493A3F85407240CC8C333C46F
:1006F000540F4420C8834004F456800146F6DFE4DA
:10070000800B0102040810204080900F87E47E01D6
:100710009360BCA3FF543F30E509541FFEE493A34C
:1007200060010ECF54C025E060A840B8E493A3FA5E
:10073000E493A3F8E493A3C8C582C8CAC583CAF0EA
:10074000A3C8C582C8CAC583CADFE9DEE780BEE5A3
:10075000245407C39406502B7F01120FCFEF24FFC0
:10076000FDEE34FFFC7F01120F9A7F01120FCF7450
:10077000002FF58274003EF583E0FDE5245407FF69
:10078000020B68E524240960280470497F01120FD8
:10079000CFEF24FFFDEE34FFFC7F01120F9A7F01A3
:1007A000120FCF74002FF58274003EF583E0F53B05
:1007B000227F01120FCFEF24FFFDEE34FFFC7F01FB
:1007C000120F9A7F01120FCF74002FF58274003E32
:1007D000F583E0F52322E5242462603D2402705A6B
:1007E000E4FF120FCF8E3C8F3DE53D2401FFE43541
:1007F0003CFED3EF94FFEE94FF40077D017F021291
:100800000E39E53D2401FDE4353CFCE4FF120F9A6E
:100810007F0C120D3D7F04801EE53B2401FFE43375
:10082000FED3EF94FFEE6480948040077D017F0249
:10083000120E39053BAF3B120D3D22E5245407FF54
:10084000C394065018120B30C0077F01120FCF74EB
:10085000002FF58274003EF583D0E0802DE524243E
:100860001160160470367F01120FCF74002FF582CD
:1008700074003EF583E53B80117F01120FCF7400B9
:100880002FF58274003EF583E523F07F01120FCF30
:10089000EF2401FDE43EFC7F01120F9A227F0E122D
:1008A0000B30C0077F01120FCF74002FF582740048
:1008B0003EF583D0E0F07F01120FCFEF2401FDE47D
:1008C0003EFC7F01120F9A7F06120B30C0077F019A
:1008D000120FCF74002FF58274003EF583D0E0F044
:1008E0007F01120FCFEF2401FDE43EFC7F01120FC8
:1008F0009A120D70AC06AD077F02020F9AE5242410
:1009000061603A2402704CE4FF120FCF8E3C8F3DA1
:10091000E53D24FFE53C34FFC3940050077D017F93
:1009200002120E39E53D24FFFDE53C34FFFCE4FFF7
:10093000120F9A7F0C120D3D7F04120D3DE53B1402
:10094000C3940050077D017F02120E39153BAF3B67
:10095000120D3D22E5242421700D120F598F3AE526
:100960003A653B603C8014120F598F3AE5245407D6
:1009700024FCFF120B30EF653A60267F02120FCF86
:10098000C006C007120F59EFFD3395E0FCD0E02DF3
:10099000FFD0E03CCF24FFFDEF34FFFC7F02020FCD
:1009A0009A7F01120F3D227F01120FCFEF24FFFD2E
:1009B000EE34FFFC7F01120F9A7F01120FCF7400FB
:1009C0002FF58274003EF583E0F53A7F01120FCFD8
:1009D000EF24FFFDEE34FFFC7F01120F9A7F01121E
:1009E0000FCF74002FF58274003EF583E0FDE53AE9
:1009F000FCED7F02020F9AE5245407FF120B30EF43
:100A000014FDE5245407FF120B68E5245407FF1278
:100A10000B30EF70267F02120FCFC006C007120FF7
:100A200059EFFD3395E0FCD0E02DFFD0E03CCF2422
:100A3000FFFDEF34FFFC7F02020F9A7F01120F3D92
:100A400022E52564016037120F01E4F521F522C388
:100A5000E5229408E521940050E77F02120FCFE5CC
:100A60002225E0243EF8E6FC08E6B50707EEB504CB
:100A7000037525010522E52270D5052180D122E5E7
:100A8000245407FFC394065005120B30800EE52452
:100A9000540724F9600B04701C120F59EF523B806D
:100AA00014E4FF120FCFAC06AD077F03120F9A902C
:100AB0000003E0523BAF3B020D3DE5245407FFC36A
:100AC00094065005120B30800EE524540724F9607B
:100AD0000B04701C120F59EF423B8014E4FF120FFD
:100AE000CFAC06AD077F03120F9A900003E0423BA4
:100AF000AF3B020D3DE5245407FFC3940650051299
:100B00000B30800EE524540724F9600B04701C128E
:100B10000F59EF623B8014E4FF120FCFAC06AD0714
:100B20007F03120F9A900003E0623BAF3B020D3D42
:100B3000AD07EDC394045012E4FF120E15EF3333EA
:100B40003354F84D242AF8E6FF22ED24FB600D14FF
:100B5000600D14600D2403700CAF2E22AF3622AF4F
:100B60002F22AF37227F0022AC07ECC3940450122F
:100B7000E4FF120E15EF33333354F84C242AF8A651
:100B80000522EC24FB600D14600D14600D2403702D
:100B90000B8D2E228D36228D2F228D37227F06122D
:100BA0000E15BF01267F02120FCFC006C007120F1D
:100BB00059EFFD3395E0FCD0E02DFFD0E03CCF2491
:100BC000FFFDEF34FFFC7F02020F9A7F01120F3D01
:100BD000227F06120E15EF70267F02120FCFC0067D
:100BE000C007120F59EFFD3395E0FCD0E02DFFD088
:100BF000E03CCF24FFFDEF34FFFC7F02020F9A7F21
:100C000001120F3D227F07120E15BF01267F02122F
:100C10000FCFC006C007120F59EFFD3395E0FCD08F
:100C2000E02DFFD0E03CCF24FFFDEF34FFFC7F023E
:100C3000020F9A7F01120F3D227F07120E15EF70EF
:100C4000267F02120FCFC006C007120F59EFFD33E7
:100C500095E0FCD0E02DFFD0E03CCF24FFFDEF3449
:100C6000FFFC7F02020F9A7F01120F3D227F0412C8
:100C70000E15EF70267F02120FCFC006C007120FAD
:100C800059EFFD3395E0FCD0E02DFFD0E03CCF24C0
:100C9000FFFDEF34FFFC7F02020F9A7F01120F3D30
:100CA000227F04120E15BF01267F02120FCFC0064D
:100CB000C007120F59EFFD3395E0FCD0E02DFFD0B7
:100CC000E03CCF24FFFDEF34FFFC7F02020F9A7F50
:100CD00001120F3D227F03120E15BF01267F021263
:100CE0000FCFC006C007120F59EFFD3395E0FCD0BF
:100CF000E02DFFD0E03CCF24FFFDEF34FFFC7F026E
:100D0000020F9A7F01120F3D227F03120E15EF7022
:100D1000267F02120FCFC006C007120F59EFFD3316
:100D200095E0FCD0E02DFFD0E03CCF24FFFDEF3478
:100D3000FFFC7F02020F9A7F01120F3D22AE07EEE9
:100D4000700A7D017F06120E391D801EEEC4540FFD
:100D50006206EE1313543F6206EEC3136206530697
:100D600001EE70047D018002E4FD7F04120E392241
:100D70007F02120FCF74002FF58274003EF583E0DE
:100D80007B00FA7F02120FCF74012FF58274003EB0
:100D9000F583E0FFEFFB7F02120F3DAE02AF0322AF
:100DA000E5242422601304701EE4FF120FCF7C00A0
:100DB000EF253BFDEC3EFC8009E4FF120FCFAC06B3
:100DC000AD077F02120F9A22EFB40A07740D120DBD
:100DD000D3740A309811A899B8130CC2983098FDB2
:100DE000A899C298B811F63099FDC299F599227F59
:100DF00002120FCFC006C007120F59EFFD3395E066
:100E0000FCD0E02DFFD0E03CCF24FFFDEF34FFFC11
:100E10007F02020F9AEFD3940740037F00227401F0
:100E20007E00A807088005C333CE33CED8F9FFEF84
:100E300055237F0060027F0122EFD39407501DED00
:100E4000700D04A807088002C333D8FC6223227403
:100E500001A807088002C333D8FC422322E52424DA
:100E6000F6600E24FE6010240470137D017F07805D
:100E70000A7D01E4FF80047D017F01120E3922E525
:100E80002424F5600E24FE600F24047012E4FD7F1C
:100E9000078009E4FDFF8004E4FD7F01120E392282
:100EA000853B3A7F07120E15EFC43333335480FF6E
:100EB000E53BC3134FF53BE53A5401FD7F07020EB6
:100EC00039E52424F160160470167F07120E15EF21
:100ED00070047D018002E4FD7F07120E39633BFF41
:100EE000227F01120FCF8E3C8F3DE4FF120FCFAC5B
:100EF00006AD077F01120F9AAD3DAC3CE4FF020F37
:100F00009A120F598F2475F003EFA42427F582E578
:100F1000F03410F583740193FA740293F902100708
:100F2000853B3A7F07120E15E53B25E04FF53BE583
:100F30003AC41313135401FD7F07020E39EFFDE588
:100F4000382DFDE433FCD3ED94FFEC6480948040B5
:100F5000020530EF2538F538227F02120FCF7400DA
:100F60002FF58274003EF583E0FE7F01120F3DAF46
:100F70000622E4F54E759850438920758DE8D28E8F
:100F8000D29912020680FB103EFFFFFFFFFFFFFF1A
:100F9000FFFFFFFFFFFFFFFFFF00AB07AF04742E53
:100FA0002BF8A607AF0574362BF8A60722E53B25DC
:100FB000E0FFE53BC413131354014FF53B22E53B1F
:100FC000C43333335480FFE53BC3134FF53B22ADAD
:100FD00007742E2DF8E6FE74362DF8E6FDEDFF229F
:100FE00010000B120FFDBF0D027F0A020DC8AF08E3
:100FF00022120D70AC06AD077F02020F9A3098FDE9
:10100000AF99C2987E00228A838982E47385233B4C
:1010100022853B2322120FE022020DC82222222227
:1010200022222222222222FF101CFF101CFF101C51
:10103000FF101CFF101CFF101CFF101CFF101CFFDA
:101040000E5DFF0E7FFF0E5DFF0E7FFF0E5DFF0E3C
:101050007FFF0EC1FF0EC1FF0EE1FF100DFF10114B
:10106000FF0003FF0003FF0003FF0003FF0003FF77
:101070000003FF0003FF0003FF0003FF0003FF0066
:1010800003FF0003FF0003FF0003FF0003FF000353
:10109000FF0003FF0003FF0003FF0003FF0003FF47
:1010A0000003FF0003FF0003FF0003FF0003FF0036
:1010B00003FF0003FF0003FF0003FF0003FF000323
:1010C000FF0003FF0003FF0003FF0003FF0003FF17
:1010D0000003FF0003FF0003FF0003FF0003FF0006
:1010E00003FF0003FF0003FF0003FF0003FF0003F3
:1010F000FF0003FF0003FF0003FF0003FF0003FFE7
:101100000003FF0003FF0003FF0003FF0003FF00D5
:1011100003FF0003FF0003FF0003FF0003FF0003C2
:10112000FF0003FF0003FF0003FF0003FF0003FFB6
:101130000003FF0003FF0003FF0003FF0003FF00A5
:1011400003FF0003FF0003FF0003FF0003FF000392
:10115000FF0003FF0003FF0003FF0003FF0003FF86
:101160000003FF0003FF0003FF0003FF0003FF0075
:1011700003FF0003FF0003FF0003FF0003FF000362
:10118000FF0003FF0003FF0003FF0003FF0003FF56
:101190000003FF0003FF0003FF0003FF0003FF0045
:1011A00003FF0003FF0003FF0A7FFF0A7FFF0A7FA0
:1011B000FF0A7FFF0A7FFF0A7FFF0A7FFF0A7FFF88
:1011C0000ABAFF0ABAFF0ABAFF0ABAFF0ABAFF0A46
:1011D000BAFF0ABAFF0ABAFF0AF5FF0AF5FF0AF5D5
:1011E000FF0AF5FF0AF5FF0AF5FF0AF5FF0AF5FF0A
:1011F0000FADFF0F20FF0FBEFF0EA0FF07D6FF08A9
:10120000FDFF07D6FF08FDFF0594FF0594FF059439
:10121000FF0594FF0594FF0594FF0594FF0594FFD7
:1012200003E5FF03E5FF03E5FF03E5FF03E5FF0338
:10123000E5FF03E5FF03E5FF0635FF0635FF06354D
:10124000FF0635FF0635FF0635FF0635FF0635FF7D
:1012500004D0FF04D0FF04D0FF04D0FF04D0FF046B
:10126000D0FF04D0FF04D0FF101DFF101DFF101D84
:10127000FF101DFF101DFF101DFF101DFF101DFF93
:10128000101EFF101EFF101EFF101EFF101EFF106D
:101290001EFF101EFF101EFF09F7FF09F7FF09F7D9
:1012A000FF09F7FF0954FF0954FF0954FF0954FFD0
:1012B0000FF1FF089DFF09A7FF101FFF0DEFFF0DA6
:1012C000A0FF0DA0FF0954FF0B9DFF0BD1FF0C05E4
:1012D000FF0C39FF0C6DFF0CA1FF0CD5FF0D09FFB2
:1012E000083BFF083BFF083BFF083BFF083BFF08AC
:1012F0003BFF083BFF083BFF074FFF074FFF074F30
:10130000FF074FFF074FFF074FFF074FFF074FFF35
:101310001020FF1021FF1022FF101CFF1023FF10D0
:0713200024FF1025FF102639
:00000001FF
